:020000040800F2
:10000000C01300204D010008D9130008870600081E
:1000100000000000000000000000000000000000E0
:100020000000000000000000000000005D16000855
:1000300000000000000000000B0100086D16000821
:100040005F010008000000005F0100085F01000878
:100050005F0100085F0100085F0100085F01000800
:1000600000000000810200085F0100085F01000835
:100070005F0100085F0100085F0100080000000048
:100080005F01000800000000000000005F010008A0
:10009000000000005D1700085F0100085F01000814
:1000A0005F0100085F0100085F010008E517000814
:1000B0005F010008000000000000000000000000D8
:1000C0000348854600F08AF800480047CD1A00082A
:1000D000C0130020084B19680868203080F3098895
:1000E000022080F31488BFF36F8F3FBCAE4608BC7C
:1000F00004BC62B61847000014000020EFF3108023
:1001000072B6704780F310887047EFF309800E4B8A
:100110001A6820381060F0C044464D4656465F4687
:10012000F0C008B572B601F0CBFF62B60CBC116826
:1001300008681030F0C8A046A946B246BB4680F316
:1001400009882038F0C81847140000200448804768
:1001500004480047FEE7FEE7FEE7FEE7FEE7FEE7AE
:100160004D170008C100000830B50B4601460020BD
:100170002022012409E00D46D5409D4205D31D46AD
:100180009540491B2546954040191546521E002DA5
:10019000F1DC30BD03460B439B0703D009E008C9DF
:1001A000121F08C0042AFAD203E00B780370401C27
:1001B000491C521EF9D27047D2B201E00270401CB5
:1001C000491EFBD270470022F6E710B513460A46D7
:1001D00004461946FFF7F0FF204610BD064C0125E6
:1001E000064E05E0E36807CC2B430C3C98471034DF
:1001F000B442F7D3FFF768FFD8230008F8230008BC
:1002000030B51B49194A02208C78131DE458240C80
:10021000240404438878C450164B144D40338C7822
:100220001448083563518C78134B2D1D63518B781E
:10023000D35801248978234353508168172291436E
:100240004205114381608168C90FFCD182680B4966
:100250000A40521C826082680A40121D8260C26895
:1002600003218A430A43C26030BD000000000240FF
:10027000C5230008002401407C000020E8FFFF7F28
:1002800010B5044800688007C00F01D000F004F8E2
:1002900010BD00000000024010B50B480221416073
:1002A0000A4C82156188511A89B2218063685918F5
:1002B0006160002100F06EFA6288218804A001F0DC
:1002C00011FB0020608010BD00000240740000207F
:1002D0002B2B2025642025640D0A0000024881682C
:1002E00002788918816070470400002010B5084822
:1002F00000240168821511430160204600F00AF8CD
:10030000002801D0012401E000F040F8204610BD93
:100310000020024000B5014687B00022152000F001
:100320005BF8152000F04CF81348026801214904DD
:100330000A43026000680840059004A9684600F07E
:100340004FF800F069F80D49FFF70EFF0D490C4A10
:100350000A600D4A401ECA6048600020086188603B
:10036000084600F070F8002802D0012007B000BD58
:10037000044800F08FF8F9E74010024040420F00B7
:100380000044014084000020E703000008B50B484A
:100390000168012211430160006810400090074885
:1003A0004038C26B01040A43C263C06B002208409C
:1003B00003210090481F00F00FF808BD40100240D4
:1003C000002805DBC106C90E0120884001490860EC
:1003D0007047000000E100E010B501F093FA10BD95
:1003E00010B5072202600A4A93685B075B0F4360FF
:1003F00093680F24240223408360926807231B0321
:100400001A40C260034800684007400F086010BDF2
:100410000010024000200240064807490068896831
:10042000064A4904490F8900515CC906C90EC840F3
:10043000704700001000002000100240A0230008B8
:1004400070477047704770B5040005D025462035C9
:10045000687F002802D006E0012070BD00202877C8
:10046000204600F016F802206877211D206801F070
:100470007DF9012240342272AA77EA7722706270F5
:10048000A270E27022716271A271E2716A7700203B
:1004900070BD7047014620314A7F012A01D00120FA
:1004A000704702224A770168CB6801221343CB6070
:1004B00000680949884202D00849884207D181680A
:1004C000074B1940062905D0DB1F994202D001686D
:1004D0001143016000207047002C014000040040DF
:1004E000070001007047000070B50446006801690C
:1004F0000025C9438907002915DBC168C94389075D
:1005000011D4E91E016101202077206880698007ED
:10051000204602D0FFF7E6FF04E000F0A7F82046EF
:1005200000F0A5F8257720680169C943490717D469
:10053000C168C943490713D40421C943016102209A
:100540002077206880698005800F204602D0FFF761
:10055000C9FF04E000F08AF8204600F088F825770B
:1005600020680169C943090716D4C168C94309074E
:1005700012D40821C9430161042020772068C06992
:100580008007204602D0FFF7ADFF04E000F06EF8D0
:10059000204600F06CF8257720680169C943C90638
:1005A00017D4C168C943C90613D41021C9430161D6
:1005B000082020772068C0698005800F204602D07F
:1005C000FFF790FF04E000F051F8204600F04FF8EC
:1005D000257720680169C943C90708D1C168C943A3
:1005E000C90704D1891E0161204600F041F8206846
:1005F0000169C943090609D4C168C943090605D47C
:100600008021C94301612046FFF71BFF2068016973
:10061000C943C90508D4C168C943090604D41249AD
:1006200001612046FFF70CFF20680169C9434906B4
:1006300009D4C168C943490605D44021C9430161B1
:10064000204600F01FF820680169C943890609D4D3
:10065000C168C943890605D42021C94301612046E8
:10066000FFF7F0FE70BD0000FFFEFFFF7047704710
:1006700010B500680249884201D1FFF72FFE10BD76
:10068000004401407047FEE770B583680022DB0735
:10069000DB0F02D00122104670BD8C684B68C56824
:1006A0002343CC68054E35402C432343C360036984
:1006B00009689B009B080B430361ECE7C73FFFFF02
:1006C000F0B5C26800230122C46852058468E407BB
:1006D000E40F02D001231846F0BDC568104C154246
:1006E00002D04D68F02D08D08E680D680F69354333
:1006F000CE683E4335434E6905E0CE680D684F69CC
:1007000035430E693E433543C66826403543C560D0
:10071000C4681442DFD04968826A0A438262DAE719
:100720003CC2FEFF10B5836AC906C90E0F248C4077
:100730009200120FA3438A401343836210BD4369A2
:1007400009028B431140490149090B43436170473A
:1007500010B543690424214007248C40A3438A40F8
:100760001343436110BD0000034A515C425801230A
:100770001A43425070470000C023000810B5044BD4
:100780005B5CC15803242403A1431143C15010BD35
:100790002B230008044B001D595C0B581B0C1B0439
:1007A00013430B5070470000C023000810B5044BE2
:1007B0005B5CC158034C21401143C15010BD000087
:1007C0002B230008EFBFFFFF10B5044B5B5CC15843
:1007D0008024A1431143C15010BD00002B23000809
:1007E00010B5044B5B5CC1580324A402A143114320
:1007F000C15010BD2B23000810B5044B5B5CC158E1
:100800002024A1431143C15010BD00002B23000838
:1008100010B5044B5B5CC1584024A1431143C15047
:1008200010BD00002B230008074B800A5840C3006E
:10083000181A0818810005480818016889098901F3
:100840001143016070470000800010000008024062
:1008500010B5044B5B5CC15803242402A14311432F
:10086000C15010BD2B230008F0B500244CE001233B
:10087000A3401A4047D04B68012B01D0022B0FD167
:100880008E688568134653435F00DF19BD43734389
:100890001D438560CB684568534395431D434560C0
:1008A0000F69C668134653435D005D19AE435F434D
:1008B0003E43C6604E68022E1FD1FF2A0ED817464F
:1008C0004A69066A94461A467A437A431701BF1A60
:1008D000BE4367467A43164306620EE0160A324666
:1008E00072434F6972437243BC461601B71A466A97
:1008F000BE4367467A43164346624A6806685343D6
:10090000AE431E430660641C0A681346E340AED142
:100910000020F0BD08B504494A6B02434A63496BA5
:100920000140009108BD00000010024008B50449D4
:100930004A6B02434A63496B0140009108BD0000C5
:100940000010024008B504494A6B02434A63496BF0
:100950000140009108BD00000010024010B504469F
:1009600000F03EFE206000F01BFE606000F028FEFC
:10097000A06010BD014610B50020032913D1134A11
:10098000516903238907890F1B041943DB43C918E5
:100990000AD001290BD0022911D000F021FE00F06D
:1009A000FFFD00F00DFE10BD00F01AFE10BD07495E
:1009B000403909684905C90FF8D0054810BDD1690B
:1009C0008907C90FFAD00120C00310BD40100240B2
:1009D0000024F40001490860704700001000002066
:1009E00070B50268174B184D984201D0A84203D148
:1009F0007024A2434C682243144E154C984208D0F0
:100A0000A84206D0134DA84203D0B04201D0A04264
:100A100004D103252D02AA43CD682A4302608A68C7
:100A2000C2620A888262984203D0B04201D0A042DA
:100A300001D109690163416901221143416100202B
:100A400070BD0000002C0140000400400044014043
:100A50000048014000200040012910D0042910D096
:100A6000102910D0402910D0CA1FF93A05D0012210
:100A7000920291420BD1052116E0042114E00021DD
:100A800012E0012110E002210EE003210CE001221E
:100A90001203914201D1062106E001221204914283
:100AA00001D1072100E00821064A1830525C1018D5
:100AB0000268044B09335B5C042199408A4302605D
:100AC0007047000019230008012910D0042910D014
:100AD000102910D0402910D0CA1FF93A05D00122A0
:100AE000920291420BD1052116E0042114E000216D
:100AF00012E0012110E002210EE003210CE00122AE
:100B00001203914201D1062106E001221204914212
:100B100001D1072100E00821064A1830525C101864
:100B20000268044B09335B5C082199400A43026068
:100B30007047000019230008F8B50D4601210C0389
:100B40002F1B0023504EA54245D007DC012D35D088
:100B5000102D37D0FF3D012D38D138E00F2424036C
:100B60003D1B67D02401A54230D1016A01252D0526
:100B7000A9430162016A446D444F3C4017683F023B
:100B80003C436F00B943178A3F053943A943958811
:100B90002D052943B04205D03D4DA84202D03D4D20
:100BA000A84207D145680126B604B5439669B60246
:100BB000354345604465D268C26561E0114600F086
:100BC0000DFC02E0114600F04DFC01465AE01146D2
:100BD00000F090FCF9E7016A01242403A1430162BB
:100BE000016A4568C46903273F02BC43274F3C4064
:100BF00017683F023C4301277F03B94317693F034E
:100C0000394301273F03B94357683F033943B04293
:100C100005D01F4EB04202D01E4EB04205D1012673
:100C2000B603B5439669B60135434560C461D268E1
:100C3000026425E0016A01252D04A9430162016ACD
:100C4000446D154F3C4017683C436F00B943178A09
:100C50003F0439439788A9433F043943B04205D044
:100C60000B4EB04202D00B4EB04205D14668AE43A7
:100C700095692D022E4346604465D268846D826575
:100C8000016219460846F8BD002C0140FF8FFFFEA7
:100C900000440140004801408FFFFEFF41680922E7
:100CA000D2029143416081682A229143816070475A
:100CB000002901D02430704728307047FEB5044623
:100CC00000680D46012738405CD12969A868EA69A7
:100CD000084369691143084321682B4A11400843BE
:100CE0002060E96860680322120390430843606053
:100CF000A969A068121190430843A0602348844268
:100D000003D10320FFF736FE06E02148844232D1AA
:100D10006846FFF723FE029800282CD06E68002E4C
:100D200029D029680027EA690B2924D80123DB038D
:100D30009A4213D109068A0D16498958FFF714FA09
:100D40004000710840183146FFF70EFA81B2124890
:100D500008400907490F0143E1600CE009068A0DCC
:100D60000C498958FFF700FA710840183146FFF71F
:100D7000FBF980B2E0602888E16A80B209090901C4
:100D80000143E1623846FEBDF369FFEF00380140E0
:100D90000044004030230008F0FF000070B592B01E
:100DA00000240C940D940E94182106A80F94FFF7BC
:100DB0000AFA18216846FFF706FA7048012102680E
:100DC00009050A4302600068084010906B49012041
:100DD00040394A6B02434A63486B6946C007C00FFB
:100DE000109001200090032001900520049400073A
:100DF000FFF73AFD0220009003200190052069468C
:100E000004940007FFF730FD5E4A5D481368052132
:100E10009B099B010B4313605B49897841585B4AEE
:100E20001140594A927881505749012589786D03BC
:100E30004158032212039143534A29439278815027
:100E40005149897841582022914311434E4A927862
:100E500081504D4989784158402291434A4A9278BD
:100E60008150494989784158802291431143464A2B
:100E700092788150444982158978415803231B0296
:100E800099431143404A927881503F49021589782D
:100E900041589B00994311433B4A927881500D94ED
:100EA0000E940F9480033A4C0C900CA92046FFF747
:100EB000EBFBE168280281430143E1602068800484
:100EC000C00FFBD025600F2100200902079106907A
:100ED000032108900A910B90099506A92046FFF777
:100EE000EFFB20694008400020612069012149078B
:100EF00088432061062200212046FFF729FC0622B4
:100F000024492046FFF724FC606804218843606080
:100F10006068082188436060A0681F49084001217B
:100F200009070843A0601E481C490068FFF71CF928
:100F3000142148430A21FFF717F900E0401E00285A
:100F4000FCD1012200212046FFF7ECFB0022012109
:100F50002046FFF7F4FB134E042132462046FFF7EC
:100F6000E1FB204601688904C90FFBD0056000221F
:100F70003146FFF7E4FB12B070BD000040100240A4
:100F8000000002400808024014230008EFBFFFFFE2
:100F90000024014004FFFF07E8FFFF7F400D03002E
:100FA000100000200200000408B50B480121826BEC
:100FB0000A438263806B0840084900900868FF225A
:100FC0001202904303229203104308600120044957
:100FD0004002086008BD00000010024008E400E084
:100FE00000E100E000B585B0142206496846FFF72D
:100FF000D1F80021684600F097FD0349086005B06C
:1010000000BD0000002300080000002010B50220F1
:10101000FFF780FC0120FFF77DFC10BD30B595B0D7
:1010200014216846FFF7CFF8202105A8FFF7CBF879
:1010300018210DA8FFF7C7F8214801210268C9034C
:101040000A43026000680024084013903F2069466C
:1010500008807D20C0001B4D029001940394284617
:10106000FFF7BEFC286880218843286001212846BC
:10107000FFF72AFD6020059006940794089405AABE
:10108000012109942846FFF757FD01212846FFF763
:10109000E3FC0120FFF74AFC10200D9002200E9087
:1010A0000420129005200F94109411940DA90007AC
:1010B000FFF7DAFB0121284600F064FA15B030BDD5
:1010C000401002400020004070B594B014216846E2
:1010D000FFF779F8202105A8FFF775F818210DA86A
:1010E000FFF771F82D480221C26B0A43C263C06B3F
:1010F0000024084013903F20694608807D20C000EE
:10110000274D0290019403942846FFF769FC286854
:101110008026B043286001212846FFF7D5FC6020D7
:10112000059006940794089405AA0121099428467D
:10113000FFF702FD01212846FFF78EFC102128460B
:10114000FFF7C2FC05AA10212846FFF7F5FC102185
:101150002846FFF781FC6868702188436860A868AA
:10116000B043A8600120FFF7E1FBC0200D900220F2
:101170000E900120129005200F94109411940DA947
:101180000007FFF771FB0121284600F0FBF9102151
:10119000284600F0F7F914B070BD000000100240BE
:1011A0000004004070B590B0202106A8FFF70BF8AE
:1011B00018216846FFF707F856480121026889039D
:1011C0000A430260006808400E900220FFF7BAFB55
:1011D00000248020504E0594022500900294039430
:1011E0000494694601953046FFF73EFB4020059484
:1011F0000090029403940494694601953046FFF7E9
:1012000033FB464D322200212846FFF70DFB00221A
:1012100011462846FFF7CAFA002211462846FFF772
:10122000ADFA202200212846FFF7E6FA00221146F7
:101230002846FFF7EDFA802200212846FFF7C4FA7E
:10124000002211462846FFF703FB002211462846DC
:10125000FFF7C6FA332201212846FFF7E5FA1022EC
:1012600001212846FFF7A2FA002201212846FFF7B4
:1012700085FA002201212846FFF7BEFA002201214B
:101280002846FFF7C5FA802201212846FFF79CFA7D
:10129000002201212846FFF7DBFA0022012128461F
:1012A000FFF79EFA1E4801680902090AC2061143A7
:1012B000016001251B49E8060860E1204002079013
:1012C0000894069409940A940C940D940C20164CDE
:1012D0000B9006A92046FFF7F1FCA068C000C008EB
:1012E000A060A068072149068843A06020686907BC
:1012F000884320602046FFF7D1FC20682843206007
:10130000E0698002C00FFBD0E0694002C00FF7D057
:1013100010B070BD401002400004005000000240B8
:1013200018E400E000E100E000380140F0B58FB0C3
:10133000202106A8FEF747FF18216846FEF743FF65
:1013400023480121C26B49040A43C263C06B0840B1
:101350000E900120FFF7F6FA00240125042005274E
:10136000059502263F070090029403946946019672
:1013700004943846FFF778FA082005950090029407
:1013800003946946019604943846FFF76DFAE1200C
:10139000400207900894069409940A940C940D94C2
:1013A0000C200C4C0B9006A92046FFF787FC20462A
:1013B000FFF774FC206828432060E0698002C00FBA
:1013C000FBD0E0694002C00FF7D00FB0F0BD0000C5
:1013D0000010024000440040FEE7000030B5026A01
:1013E000520852000262026A43688469194DA408D7
:1013F000A4002C400D682C430225AA430D692A4302
:1014000052084D6852002A43134DA84205D0134D8F
:10141000A84202D0124DA84214D10825AA434D6912
:10142000AD002A430425AA438D68AD002A43FF2559
:101430000135AB438D692B4301256D02AB43CD696B
:101440006D002B4343608461C968416302620020E0
:1014500030BD00008FFFFEFF002C01400044014022
:101460000048014070B5026A1025AA430262026A70
:101470004368846903263602B4431A4E34400E682A
:10148000360234432026B2430E6936013243AA4362
:101490004D682D012A43144DA84205D0134DA84292
:1014A00002D0134DA84215D18025AA434D69AD0144
:1014B0002A434025AA438D68AD012A430125AD0288
:1014C000AB438D69AD002B430125ED02AB43CD69E4
:1014D000ED002B4343608461C96881630262002090
:1014E00070BD0000FF8FFFFE002C01400044014052
:1014F0000048014070B5026AFF250135AA43026227
:10150000026A4368C4691B4EA408A40034400E68F4
:1015100034436E00B2430E6936023243AA434D682B
:101520002D022A43144DA84205D0144DA84202D0E2
:10153000134DA84217D10125ED02AA434D69AD0212
:101540002A430125AD02AA438D68AD022A43012535
:101550002D03AB438D692D012B4301256D03AB4357
:10156000CD696D012B434360C461C968C1630262E8
:10157000002070BD8FFFFEFF002C014000440140A1
:1015800000480140026A0A430262416C0122D20310
:10159000114341640168012211430160704700005A
:1015A000054989688A093C210A400A400349895C47
:1015B000C906C90EC84070470010024060230008E9
:1015C00005498968054A4904490F8900515CC906E3
:1015D000C90EC8407047000000100240A023000858
:1015E00010B50B4988683822104008280AD0102806
:1015F0000AD0086801218004400F81400548FEF7A9
:10160000B3FD10BD044810BD00F008F810BD000087
:10161000001002400024F40000127A0010B50D4AB8
:10162000D0680D498007800F022802D0032800D11E
:101630004910D068440FD0684006430FD068641C3E
:101640004004400E4843591CFEF78EFD2146FEF72C
:101650008BFD10BD001002400024F4007047FF24F1
:10166000F534204600F053FAFBE7000010B5FEF712
:1016700045FD044600F090FD002803D001200349F9
:10168000000748602046FEF73DFD10BD00ED00E07C
:1016900010B5294802210268D208D2000A4302602C
:1016A00001684907490F0229FAD1244801688215C7
:1016B0001143016001684905C90FFBD02049C26888
:1016C000204B1A401143C1600168012212061143E8
:1016D0000160C16812011143C16001688901C90F2D
:1016E000FBD081680F22120291438160826802213F
:1016F000D208D2000A438260382281681140102942
:10170000FBD1816807221203914381600E48FFF7E5
:1017100061F90020FEF7FEFD002801D072B6FEE759
:101720000648403041698908890041614169890062
:101730008908416110BD00000020024000100240F5
:10174000020800208C80FF1F0090D0030120024976
:10175000C00688607047000000ED00E010B5024848
:10176000FEF7C2FE10BD00008400002070B50268C4
:10177000174B184E984201D0B04203D17024A243B7
:101780004C682243144C154D984208D0B04206D004
:10179000134EB04203D0A04201D0A84204D1032688
:1017A0003602B243CE6832438026B2434E6932439A
:1017B00002608A68C2620A688262984203D0A042CC
:1017C00001D0A84201D1096901630121416170BDC5
:1017D000002C01400004004000440140004801404A
:1017E0000020004010B50448C069C006C00F01D0F9
:1017F00000F04AF810BD000000380140F8B51F4D58
:101800001C4F29781B4E1C480C37C8511C4C012119
:101810002046FFF74DFA2A78391F50508A150021CB
:101820003046FEF7B7FF69781648C85100212046B8
:10183000FFF73EFA6A78391F50508A150121304669
:10184000FEF7A8FFA06840210843A060A06880219F
:101850000843A06020681021084320602878305891
:10186000022108432978705000213046FEF77CFFA2
:10187000F8BD000000000240C00D0020C023000899
:1018800000380140C00E002070B50F4910200862DA
:101890000F480E4E0078311D40588D150D4C291AF9
:1018A0006088091A89B24018218083B26380606819
:1018B000421809A0626000F015F82A46002130465F
:1018C000FEF768FF002070BD0038014000000240B4
:1018D000C0230008740000202564202564202564AE
:1018E0000D0A00000FB410B503A9044B044A029876
:1018F00000F03AF810BC08BC04B01847B91A000848
:10190000800000208307FF22DB0E9A408907090E22
:101910009940002808DB830809489B001B181868B9
:1019200090430843186070470007000F0838830889
:1019300004489B001B18D86990430843D86170473E
:1019400000E400E000ED00E002E008C8121F08C15A
:10195000002AFAD170477047002001E001C1121F30
:10196000002AFBD170470000FFB58DB0044600256A
:1019700006E025280AD0109A0F999047641C6D1C28
:1019800020780028F5D1284611B0F0BD00270121AC
:10199000484A009700E00743641C23780846203B30
:1019A00098401042F7D120782E2817D10420074301
:1019B0006078641C2A280CD10E98641C02C800911F
:1019C0000E900BE000990A22514330394018641CF4
:1019D00000902078014630390929F3D92078002871
:1019E000D1D0642808D0692806D075281ED0109A56
:1019F0000F9990476D1C5BE00A200E99019001C978
:101A00000E91002802DA40422D2102E0390504D56A
:101A10002B216A461172012103E0F90704D020212D
:101A2000F7E70BAE0B910DE00021FAE70A200E99C3
:101A3000019001C90E91F7E70199FEF795FB30314E
:101A4000761E31700028F7D103A8801B203001904A
:101A5000780701D5009801E00120009001998842A3
:101A600001DD401A00E000200027009006E002A8F7
:101A7000109AC05D0F9990476D1C7F1C0B98874290
:101A8000F5DB04E0109A30200F9990476D1C009907
:101A9000481E00900029F5DC05E03078109A761C8D
:101AA0000F9990476D1C0199481E01900029F4DCA4
:101AB000641C65E7092801000349C2B28A62CA6949
:101AC0001206D20FFBD0704700440040FEF70EFC18
:101AD000FFF7DEFDFFF79AFAFFF766FAFFF75EF908
:101AE000FFF7F2FAFFF79AFAFFF75CFBFFF71EFC2D
:101AF000FFF784FEFEF784FBFFF774FA00F00FF89F
:101B0000FEE701460020842900D0C81C704710B5AC
:101B1000002800D1012000F08DFA002010BD10B582
:101B200000F0A0FA002010BD3EB5044608200D4686
:101B3000205EFFF7E6FF02A901910090208A2B4664
:101B400082B22168606800F0FFFA012801D000200D
:101B50003EBD02983EBD0000F8B5134C0F46E66846
:101B600005462068001D00F0C1F9681C07D1002F50
:101B700005D021680D48091D00F0F1F9F8BD206875
:101B8000751945602168B54204D2A06B091D00F0AB
:101B9000CEF9F8BD606B091D00F0C9F9A06A854255
:101BA000F7D2A562F8BD000014000020AC010020AF
:101BB000F8B5054600F0E0F9294CA068401CA0608B
:101BC0002068284F002803D06069002827D02CE027
:101BD0002560A068012828D1002614207043C01970
:101BE00000F097F9761C072EF7D31E488C3000F0D2
:101BF00090F91C48A03000F08CF91A48B43000F07D
:101C000088F91848C83000F084F91648DC3000F034
:101C100080F914488C3060631430A06305E02068BC
:101C2000E96AC06A884200D82560606A401C606228
:101C3000E86A2169884200D9206114214843C0190B
:101C4000291D00F08CF900F0A3F96069002806D086
:101C50002068E96AC06A884201D200F0DFF9F8BD65
:101C600014000020D000002010B50446006B00F0E6
:101C70009DF9204600F09AF910BD000003210E489E
:101C80008902420705D0C01DC0080B4AC000821A55
:101C9000891A0A4A0023411809C20839C908C9002B
:101CA000203A11604B600B600B1A0AC09360012050
:101CB000C007536050617047C001002068000020D9
:101CC0000F4E104C3746C83F11E000F055F9F06850
:101CD000C568281D00F00AF9A068401EA060606871
:101CE000401E606000F054F92846FFF7BDFF6068B1
:101CF0000028EAD138680128F9D900F08FF9F6E711
:101D00009801002014000020FFB581B00C9C9000C9
:101D1000236B001F1818C7080A9DFF00780701D021
:101D200072B6FEE72646403600290DD00020231863
:101D30000A5C20331A750A5C002A02D0401C102865
:101D4000F5D30020F07002E0002034210855072D63
:101D500000D30625E56200206564A064201D00F024
:101D6000E3F82046183000F0DFF824610720401B1C
:101D70006462A0610020E06430743846049A0199DE
:101D800000F0A4F820600B98002800D0046005B093
:101D9000F0BD000030B5114900E011460A688242EA
:101DA000FBD34B685C18844203D140681818486024
:101DB000084643681C18944209D1084C183C246812
:101DC000A24209D052689A1842600A6812680260FA
:101DD000814200D0086030BD0460F9E7680000204F
:101DE0000648416B0968002905D0416BC968C9687C
:101DF0004968816270470021C943FAE71400002056
:101E000003480068401C72B600D0FEE7FEE7000001
:101E100070000020F8B50546002700F049F92A4E69
:101E20003068002801D1FFF729FF7069054242D1CF
:101E3000002D40D00835680708D06807400F0821FA
:101E4000081A4519680701D072B6FEE7002D32D096
:101E5000706885422FD81C48183001460C6801E094
:101E600020460C466168A94202D221680029F7D1B8
:101E700031688C421FD007682168016060680837AC
:101E8000411B102908D96019420701D072B6FEE73C
:101E900041606560FFF77EFF61687068401A70609E
:101EA000B268904200D2B06070690143002003C460
:101EB000F068401CF06000F0CDF9780701D072B6F0
:101EC000FEE73846F8BD00005000002010B50124A0
:101ED000031F24061C601B1F1960191F024B0B6097
:101EE000143940380A6010BD011E0008436882683A
:101EF00001699A60836842685A604A68824201D1E7
:101F000082684A60002202610868401E0860086812
:101F100070470146083100224160D243C1608260AF
:101F2000016100210160704700210161704730B5F7
:101F30000B685A1C02D00246083202E0026904E033
:101F40002246546825689D42FAD953684B609960CF
:101F50008A60516008610168491C016030BD4268B7
:101F60004A6093688B60936859609160086101686A
:101F7000491C01607047000072B604480168491CA2
:101F80000160BFF34F8FBFF36F8F70477000002069
:101F900005490868002804D0401E086000D162B6D8
:101FA000704772B6FEE700007000002070B5002890
:101FB0001DD004460E4D083C60686969084201D195
:101FC00072B6FEE72268002A01D072B6FEE78843A7
:101FD000606000F06DF860686968401868602046CD
:101FE000FFF7D8FE2869401C286100F033F970BD66
:101FF0005000002010B5074C00202061A061064869
:102000007D21C9000068FEF7AFF8401E606107201F
:10201000206110BD00E000E0100000200120044914
:1020200000074860BFF34F8FBFF36F8F704700000A
:1020300000ED00E010B502000FD00948006B002849
:1020400001D072B6FEE700F033F800211046FFF72A
:1020500083FD00F0FFF8002801D1FFF7DFFF10BD7E
:10206000140000201CB50E48002401902346802255
:102070000CA100940D4800F067F8012803D0401C23
:102080000CD172B6FEE772B600210548C9432C3860
:10209000816201214161C46000F03EF81CBD000076
:1020A0004000002049444C4500000000C11C0008CD
:1020B0000248016B491C01637047000014000020B6
:1020C00010B51348016B002902D00121C16110BD78
:1020D0000021C16101690F4A02E0002915D0491EA3
:1020E00014234B43D358002BF7D014234B439A1897
:1020F000536814465B6808345360A34201D15B689F
:102100005360DA680260016110BD72B6FEE700003C
:1021100014000020D000002010B50948016AFF22F9
:10212000120411430162016A120211430162FFF7B6
:1021300061FF044900200860FDF7CCFF002010BDBE
:1021400000ED00E070000020FFB585B0164690005D
:102150000F9FFFF75FFE05001AD05420FFF75AFECD
:10216000040012D0256300210E980391019700907E
:1021700002943246089B06990598FFF7C5FD204654
:10218000FFF716FD012009B0F0BD2846FFF70EFF4E
:102190000020C043F7E70000F8B52C4C0027206B67
:1021A000002804D0A069401CA0613846F8BDE6684C
:1021B000761CE6600ED1606B0068002801D072B614
:1021C000FEE7606BA16B6163A063206A401C206224
:1021D000FFF706FEA06A86420AD3606B00680028FB
:1021E00014D0606BC068C5686868864211D2A0626E
:1021F00020681421C06A484315490858012800D9AD
:102200000127E0690028D0D00127CEE70020C04395
:10221000EDE7281DFFF76AFEA86A002803D02846CC
:102220001830FFF763FEE86A2169884200D920610F
:102230001421484306494018291DFFF790FEE86A1B
:102240002168C96A8842C8D30127C6E71400002064
:10225000D0000020F8B5284C0025206B2E46002821
:1022600008D0FFF789FE206B401E2063206B0028FA
:1022700002D03DE072B6FEE7A168204F00291DD1D3
:1022800036E0F868C56828461830FFF72FFE281D8D
:10229000FFF72CFEE86A2169884200D920611421E9
:1022A00048431649B4394018291DFFF758FEE86A1B
:1022B0002168C96A884201D30120E061386800289A
:1022C000DFD1002D01D0FFF78BFDA569002D09D0CE
:1022D0000127FFF761FF002800D0E7616D1EF8D1EC
:1022E0000020A061E069002802D00126FFF796FED9
:1022F000FFF74EFE3046F8BD140000208401002098
:10230000CC2300085F160008000000000000000059
:1023100080000000081C3044580000000004040441
:102320003C3C000008000000080008081C3044582D
:102330000100000002000000040000000600000090
:10234000080000000A0000000C000000100000005F
:10235000200000004000000080000000000100009C
:10236000000000000000000000000000000000006D
:10237000000000000000000000000000000000005D
:102380000100000002000000030000000400000043
:10239000060000000700000008000000090000001F
:1023A000000000000000000000000000000000002D
:1023B0000100000002000000030000000400000013
:1023C000081C304458081C3044580000646566619D
:1023D000756C745461736B00F823000800000020D2
:1023E00084000000481900087C24000884000020B4
:1023F0003C13000058190008000000000100000014
:1024000004000000000000000024F40000000000B0
:1024100000000000000000000000000000000000BC
:1024200000000000000000000000000000000000AC
:10243000000000000000000000000000000000009C
:10244000000000000000000000000000000000008C
:10245000000000000000000000000000000000007C
:102460000000000000000000AAAAAAAA00000000C4
:0C24700000000000000000000000000060
:04000005080000C12E
:00000001FF
